:100000007128210820040319A00A8030201AA106B3
:100010002019A106A018A106210DA00DA10D6C2884
:10002000A301A200FF30A207031CA307031C6C2836
:100030000330A100DF301E201228A101E83EA000FD
:10004000A109FC30031C2728A00703182428A007B7
:100050006400A10F242820182D28A01C312800009E
:1000600031280800A20002304028A20001304028B8
:10007000A20006304028A20004304028A20005302B
:10008000A80023082102031D47282208200204306B
:1000900003180130031902302805031DFF306C28B6
:1000A000A501A4011030A600210DA40DA50D220864
:1000B000A4022308031C230FA502031866282208A4
:1000C000A40723080318230FA5070310A00DA10DF3
:1000D000A60B542820086C28831303138312640092
:1000E00008008316870185018312D801D9015808B9
:1000F000A0005908A100A30100308A013E208A1106
:10010000031D84288A11EF22D80A0319D90A44084A
:10011000A0004508A1008A0101202008C400210890
:10012000C5004408A0004508A1001330A200A301A7
:100130008A0150202408C6002508C7000130460760
:10014000C80047080318013EC9004608A000470838
:10015000A100A30101308A013E208A11031DB428A9
:100160008A1102258A11ED2A4608A0004708A1003D
:10017000A30102308A013E208A11031DC3288A157B
:10018000D2248A11ED2A4608A0004708A100A30145
:1001900003308A013E208A11031DD2288A112A25A4
:1001A0008A11ED2A4608A0004708A100A3010430E7
:1001B0008A013E208A11031DE1288A11B7268A117F
:1001C000ED2A4608A0004708A100A30105308A01D6
:1001D0003E208A11031D04290130D600D70156089C
:1001E000A0005708A100A3010A308A0135208A1116
:1001F000031D02298A11EE27D60A0319D70A8A118C
:10020000031DEF288A11ED2A4608A0004708A10027
:10021000A30106308A013E208A11031D5E29831640
:1002200050088312A000831651088312A1008A018E
:10023000012020088316D000831221088316D100E4
:1002400050088312A000831651088312A1001030B9
:10025000A200A3018A01502024088316D200831231
:1002600025088316D30004305207D400530803181E
:10027000013ED5000130D600D701831283165608FF
:100280008312A000831657088312A1008316550815
:100290008312A3008316540883128A0135208A1121
:1002A000031D5C298A157A208316D60A0319D70AFA
:1002B0008A118312031D3E298A11ED2A4608A000E7
:1002C0004708A100A30107308A013E208A11031DBF
:1002D000B829831650088312A00083165108831290
:1002E000A1008A01012020088316D0008312210872
:1002F0008316D10050088312A00083165108831280
:10030000A1001030A200A3018A0150202408831606
:10031000D200831225088316D30004305207D4007C
:1003200053080318013ED5000130D600D7018312CF
:10033000831656088312A000831657088312A10063
:10034000831655088312A3008316540883128A016A
:1003500035208A11031DB6298A15B2208316D60AC4
:100360000319D70A8A118312031D98298A11ED2ACD
:100370004608A0004708A100A30108308A013E20DA
:100380008A11031DC7298A15B1238A11ED2A46084F
:10039000A0004708A100A30109308A013E208A116C
:1003A000031DD6298A1533248A11ED2A4608A00098
:1003B0004708A100A3010A308A013E208A11031DCB
:1003C000E5298A156C238A11ED2A4608A000470802
:1003D000A100A3010B308A013E208A11031DF429DC
:1003E0008A154D218A11ED2A4608A0004708A10070
:1003F000A3010C308A013E208A11031D1F2A831697
:100400000130D800D9018312831658088312A00046
:10041000831659088312A100A3010A308A013520EE
:100420008A11031D1D2A8A15D3218316D80A0319A0
:10043000D90A8A118312031D042A8A11ED2A46085B
:10044000A0004708A100A3010E308A013E208A11B6
:10045000031D2E2A8A1519228A11ED2A4608A000AA
:100460004708A100A3010F308A013E208A11031D15
:100470008E2A9030E6000130E7006608A000670889
:10048000A100A30196308A013B208A11031D582A3E
:100490008A1590273230E60200308A110318542A58
:1004A000013E8A110318582AE7028A1103183D2ACF
:1004B0009630E600E7016608A0006708A100A301E6
:1004C0005A308A013B208A11031D762A8A1590270B
:1004D0000A30E60200308A110318722A013E8A119E
:1004E0000318762AE7028A1103185B2A0130E60016
:1004F000E7016608A0006708A100A30107308A0190
:1005000035208A11031D8C2A8A159027E60A0319C3
:10051000E70A8A11031D792A8A11ED2A4608A000EC
:100520004708A100A30110308A013E208A11031D53
:10053000C12A83166E30A200A301831283162208FB
:100540008312A000831623088312A100A301503058
:100550008A013B208A11031DBF2A8A15A2220A3074
:100560008316A20200308A1183120318BB2A013EAF
:100570008A110318BF2AA3028A1103189E2A8A111E
:10058000ED2A4608A0004708A100A30111308A0106
:100590003E208A11031DD02A8A1554258A11ED2A7E
:1005A0004608A0004708A100A30113308A013220A9
:1005B0008A11031DE62A4608A0004708A100A301EE
:1005C00012308A013E208A11031DED2A8A157226F7
:1005D0006508A30064088A0111208A017728831620
:1005E0001930C200C3018312831642088312A0008F
:1005F000831643088312A1000B30A300B8308A0190
:1006000035208A11031D452B0130BE00BF013E0875
:10061000A0003F08A100A30102308A0135208A1101
:10062000031D382B3F3087000730850083164308B1
:100630008312A1008316420883128A011E208701BB
:10064000850183164208883CEC004308031C013EE8
:10065000133CED006D088312A10083166C08831211
:100660008A011E20BE0A0319BF0A8A11031D072B27
:1006700019308316C2078A118312031CF42A8316C9
:10068000C30A8A118312031DF42A8316B830C200EC
:100690000B30C3008312831642088312A000831616
:1006A00043088312A1001130A30094308A01352041
:1006B0008A11031D9C2B0130BE00BF013E08A00023
:1006C0003F08A100A30102308A0135208A11031DD1
:1006D0008F2B3F3087000730850083164308831235
:1006E000A1008316420883128A011E20870185011A
:1006F00083164208883CEC004308031C013E133C6F
:10070000ED006D088312A10083166C0883128A0124
:100710001E20BE0A0319BF0A8A11031D5E2B0A3070
:100720008316C2078A118312031C4B2B8316C30A3C
:100730008A118312031D4B2B83169430C200113093
:10074000C3008312831642088312A0008316430855
:100750008312A1001330A30088308A0135208A114A
:10076000031DF32B0130BE00BF013E08A0003F086F
:10077000A100A30102308A0135208A11031DE62B56
:100780003F30870007308500831643088312A1009D
:100790008316420883128A011E2087018501831671
:1007A0004208883CEC004308031C013E133CED006A
:1007B0006D088312A10083166C0883128A011E2023
:1007C000BE0A0319BF0A8A11031DB52B0530831613
:1007D000C2078A118312031CA22B8316C30A8A1133
:1007E0008312031DA22B080083168830DC0013300F
:1007F000DD00831283165C088312A00083165D0857
:100800008312A1001130A30094308A013B208A1189
:10081000031D4E2C0130C200C3014208A000430852
:10082000A100A30102308A0135208A11031D3E2C4C
:100830003F3087000730850083165D088312A100D2
:1008400083165C0883128A011E2087018501883087
:1008500083165C07EE0013300318013E5D07EF00BE
:100860006F088312A10083166E0883128A011E206E
:10087000C20A0319C30A8A11031D0D2C23308316E3
:10088000DC0200308A11831203184A2C013E8A11BF
:1008900003184E2CDD028A110318FA2B83169430AC
:1008A000DC001130DD00831283165C088312A00087
:1008B00083165D088312A1000730A300D0308A019F
:1008C0003B208A11031DA82C0130C200C30142083D
:1008D000A0004308A100A30102308A0135208A113B
:1008E000031D982C3F3087000730850083165D0874
:1008F0008312A10083165C0883128A011E208701DF
:100900008501883083165C07EE0013300318013E22
:100910005D07EF006F088312A10083166E08831233
:100920008A011E20C20A0319C30A8A11031D672CFB
:1009300014308316DC0200308A1183120318A42CB1
:10094000013E8A110318A82CDD028A110318542CC9
:100950008316D030DC000730DD00831283165C087C
:100960008312A00083165D088312A100A30100304A
:100970008A013B208A11031D012D0130C200C301F1
:100980004208A0004308A100A30102308A013520DB
:100990008A11031DF12C3F30870007308500831634
:1009A0005D088312A10083165C0883128A011E2051
:1009B00087018501883083165C07EE001330031829
:1009C000013E5D07EF006F088312A10083166E08D9
:1009D00083128A011E20C20A0319C30A8A11031D49
:1009E000C02C0A308316DC0200308A1183120318EF
:1009F000FD2C013E8A110318012DDD028A11031816
:100A0000AE2C08000130FE00FF017E08A0007F0828
:100A1000A100A3010A308A0135208A11031D292D66
:100A20003230EA00EB013F308700073085006B0869
:100A3000A3006A088A011120870185016B08A300C1
:100A40006A088A011120FE0A0319FF0A8A11031D90
:100A5000052D080083169630A000A101831283168D
:100A600020088312A000831621088312A100A3018D
:100A700064308A013B208A11031D502D8A1195256F
:100A80000F308316A00200308A11831203184C2DF8
:100A9000013E8A110318502DA1028A1103182F2D2F
:100AA00083166430A000A1018312831620088312EC
:100AB000A000831621088312A100A3011E308A0121
:100AC0003B208A11031D762D8A1195250A30831645
:100AD000A00200308A1183120318722D013E8A1180
:100AE0000318762DA1028A110318552D83160130A3
:100AF000BA00BB01831283163A088312A000831642
:100B00003B088312A100A30107308A0135208A1116
:100B1000031D942D8A1195258316BA0A0319BB0A61
:100B20008A118312031D7B2D0800243087000430B6
:100B30008500831621088312A300831620088312E0
:100B40008A011120103087000230850083162108A9
:100B50008312A3008316200883128A0111208701C3
:100B600001308500831621088312A3008316200814
:100B700083128A0111200930870001308500831615
:100B800021088312A3008316200883128A011120F2
:100B90001030870002308500831621088312A300DD
:100BA0008316200883128A011120870104308500F2
:100BB000831621088312A3008316200883128A015A
:100BC0001120870107308500831621088312A300B6
:100BD0008316200883128A011120183087008501AE
:100BE000831621088312A3008316200883128A012A
:100BF0001120013087008501831621088312A3008C
:100C00008316200883128A0111200730870085018E
:100C1000831621088312A3008316200883128A01F9
:100C20001120183087008501831621088312A30044
:100C30008316200883128A01112087010130850064
:100C4000831621088312A3008316200883128A01C9
:100C50001120093087000130850083162108831296
:100C6000A3008316200883128A0111201230870006
:100C70008501831621088312A3008316200883129E
:100C80008A01112004308700831621088312A300F3
:100C90008316200883128A01112024308700043033
:100CA0008500831621088312A3008316200883126F
:100CB0008A011120123087008501831621088312D2
:100CC000A3008316200883128A01112001308700B7
:100CD000831621088312A3008316200883128A0139
:100CE0001120073087008501831621088312A30095
:100CF0008316200883128A01112030308700831662
:100D000021088312A3008316200883128A01112070
:100D1000870104308500831621088312A3008316FF
:100D2000200883128A0111200730850083162108CC
:100D30008312A3008316200883128A011120303009
:100D400087008501831621088312A30083162008DB
:100D500083128A01112064308700831621088312D0
:100D6000A3008316200883128A011120080083162D
:100D7000C830B200B3018312831632088312A00078
:100D8000831633088312A100A30164308A013B203B
:100D90008A11031DDD2E8A11F42614308316B20247
:100DA00000308A1183120318D92E013E8A110318CC
:100DB000DD2EB3028A110318BC2E0130CC00CD0108
:100DC0004C08A0004D08A100A30107308A0135207E
:100DD0008A11031DF32E8A11F426CC0A0319CD0AB9
:100DE0008A11031DE02E080083165030A600A701CB
:100DF0008312013087008501831627088312A30020
:100E00008316260883128A0111200A308700831670
:100E100027088312A3008316260883128A01112053
:100E20001430870001308500831627088312A30041
:100E30008316260883128A01112020308700023091
:100E40008500831627088312A300831626088312C1
:100E50008A01112087010430850083162708831238
:100E6000A3008316260883128A011120043087000C
:100E70008501831627088312A30083162608831290
:100E80008A01112022308700831627088312A300CD
:100E90008316260883128A0111201130870004303E
:100EA0008500831627088312A30083162608831261
:100EB0008A01112008308700023085008316270838
:100EC0008312A3008316260883128A01112087014A
:100ED00001308500831627088312A3008316260895
:100EE00083128A01112087010430850083162708A8
:100EF0008312A3008316260883128A011120203052
:100F0000870002308500831627088312A30083160A
:100F1000260883128A0111201430870001308500D1
:100F2000831627088312A3008316260883128A01DA
:100F300011200A3087008501831627088312A30039
:100F40008316260883128A01112001308700831638
:100F500027088312A3008316260883128A01112012
:100F6000870101308500831627088312A3008316AA
:100F7000260883128A01112008308700023085007C
:100F8000831627088312A3008316260883128A017A
:100F90001120113087000430850083162708831242
:100FA000A3008316260883128A01112022308700AD
:100FB0008501831627088312A3008316260883124F
:100FC0008A01112004308700831627088312A300AA
:100FD0008316260883128A011120080083165030D8
:100FE000A800A90183124008A0004108A100A301A4
:100FF00000308A013E208A15031D0228093087002F
:10100000013085004008A0004108A100A301003084
:101010008A0138208A15031D11280F3087000130FE
:101020008500C00A0319C10A831629088312A30088
:101030008316280883128A0111201230870002309B
:101040008500831629088312A300831628088312BB
:101050008A01112027308700043085008316290873
:101060008312A3008316280883128A0111203830C6
:1010700087008501831629088312A3008316280898
:1010800083128A01112024308700073085008316DF
:1010900029088312A3008316280883128A011120CD
:1010A0001230870002308500831629088312A300BE
:1010B0008316280883128A0111200930870007301F
:1010C0008500831629088312A3008316280883123B
:1010D0008A01112038308700850183162908831280
:1010E000A3008316280883128A0111200730870085
:1010F0008501080083166430AA00AB018312033017
:1011000087000630850083162B088312A300831600
:101110002A0883128A01112038308700850183163E
:101120002B088312A30083162A0883128A01112038
:10113000063087000330850083162B088312A30036
:1011400083162A0883128A0111203830870085010E
:1011500083162B088312A30083162A0883128A01A0
:10116000112008006430FA00FB01023087000530CE
:1011700085007B08A3007A088A0111203830870097
:1011800085017B08A3007A088A01112005308700B9
:10119000023085007B08A3007A088A0111203830CC
:1011A000870085017B08A3007A088A0111200800C6
:1011B00083163C30A400A5018312850187018316A4
:1011C00025088312A3008316240883128A011120A4
:1011D00004308700831625088312A3008316240891
:1011E00083128A011120023087008316250883129A
:1011F000A3008316240883128A011120013087007E
:10120000831625088312A3008316240883128A01FB
:10121000112020308700831625088312A30083162F
:10122000240883128A0111201030870083162508B4
:101230008312A3008316240883128A011120083028
:101240008700831625088312A300831624088312BF
:101250008A01112004308500870183162508831236
:10126000A3008316240883128A011120023085000E
:10127000831625088312A3008316240883128A018B
:10128000112001308500831625088312A3008316E0
:10129000240883128A01112008008230EC00ED013D
:1012A0006C08A0006D08A100A30164308A013B20F6
:1012B0008A15031D6B298A15A8210A30EC0200301B
:1012C0008A1503186729013E8A1503186B29ED0258
:1012D0008A15031850296430EC00ED016C08A00059
:1012E0006D08A100A3014B308A013B208A15031D24
:1012F00089298A15A8210530EC0200308A150318C7
:101300008529013E8A1503188929ED028A150318DB
:101310006E2983160130BE00BF01831283163E087A
:101320008312A00083163F088312A100A3010A3094
:101330008A0135208A15031DA7298A15A82183163D
:10134000BE0A0319BF0A8A158312031D8E290800DD
:101350002030870085016D08A3006C088A011120E8
:1013600014308700043085006D08A3006C088A01E2
:1013700011200A308700023085006D08A3006C0838
:101380008A01112001308700013085006D08A3001B
:101390006C088A011120870185016D08A3006C0883
:1013A0008A01112008005030EE00EF01870104305F
:1013B00085006F08A3006E088A01112002308500A5
:1013C0006F08A3006E088A0111200830870085018C
:1013D0006F08A3006E088A011120203087006F0873
:1013E000A3006E088A011120103087006F08A30047
:1013F0006E088A011120013087006F08A3006E0873
:101400008A011120043087006F08A3006E088A014A
:101410001120023087006F08A3006E088A01112096
:101420000130850087016F08A3006E088A01112032
:1014300008001E30F200F3017208A0007308A1003A
:10144000A30132308A0135208A15031D5D2A02303E
:10145000850087017308A30072088A0111201030EB
:10146000870085017308A30072088A0111200230E9
:1014700087007308A30072088A01112005308700D5
:101480007308A30072088A011120283087007308AE
:10149000A30072088A0111208701053085007308B6
:1014A000A30072088A0111200530F2078A15031C77
:1014B0001C2AF30A8A15031D1C2A3230F200F3019C
:1014C0007208A0007308A100A30164308A013520CE
:1014D0008A15031DA12A0230850087017308A30025
:1014E00072088A0111201030870085017308A3005B
:1014F00072088A011120023087007308A300720865
:101500008A011120053087007308A30072088A0140
:101510001120283087007308A30072088A01112067
:101520008701053085007308A30072088A01112025
:101530000A30F2078A15031C602AF30A8A15031D74
:10154000602A08000430870085018316230883126F
:10155000A3008316220883128A01112024308700F9
:10156000831623088312A3008316220883128A019C
:10157000112004308500831623088312A3008316EC
:10158000220883128A011120063085008316230861
:101590008312A3008316220883128A0111202030AF
:1015A000870007308500831623088312A300831663
:1015B000220883128A01112008308700831623082D
:1015C0008312A3008316220883128A011120093096
:1015D000870003308500831623088312A300831637
:1015E000220883128A0111200B3087000130850008
:1015F000831623088312A3008316220883128A010C
:1016000011201B3087008501831623088312A30055
:101610008316220883128A011120133087000230BA
:101620008500831623088312A300831622088312E1
:101630008A011120123087000630850083162308A6
:101640008312A3008316220883128A0111203030EE
:10165000870006308500831623088312A3008316B3
:10166000220883128A011120243087000630850069
:10167000831623088312A3008316220883128A018B
:10168000112004308500831623088312A3008316DB
:10169000220883128A0111208501831623088312F0
:1016A000A3008316220883128A01112004308700C8
:1016B000831623088312A3008316220883128A014B
:1016C00011208701831623088312A30083162208A2
:1016D00083128A0111200800F430DA000130DB00A7
:1016E000053085003D3087005B08A3005A088A0159
:1016F0001120850187015B08A3005A088A01112087
:10170000053085002A3087005B08A3005A088A014B
:101710001120850187015B08A3005A088A01112066
:1017200002308500173087005B08A3005A088A0141
:101730001120850187015B08A3005A088A01112046
:1017400002308500173087005B08A3005A088A0121
:101750001120850187015B08A3005A088A01112026
:1017600008004B30DC00DD010130850087015D0899
:10177000A3005C088A011120013085001030870029
:101780005D08A3005C088A01112001308500143037
:1017900087005D08A3005C088A011120850187018C
:1017A0005D08A3005C088A011120013085008701D3
:1017B0005D08A3005C088A01112003308500083011
:1017C00087005D08A3005C088A01112003308500B2
:1017D0002A3087005D08A3005C088A0111200330CD
:1017E00085002E3087005D08A3005C088A01112067
:1017F000850187015D08A3005C088A011120013082
:10180000850087015D08A3005C088A011120033070
:101810008500083087005D08A3005C088A0111205C
:1018200007308500093087005D08A3005C088A0145
:101830001120073085002B3087005D08A3005C086D
:101840008A011120073085002F3087005D08A30032
:101850005C088A011120850187015D08A3005C08EE
:101860008A011120080083166430D800D901831240
:10187000043085008701831659088312A30083165C
:10188000580883128A011120043085000230870035
:10189000831659088312A3008316580883128A01FD
:1018A0001120013085000930870083165908831202
:1018B000A3008316580883128A0111200430850082
:1018C0008701831659088312A300831658088312D0
:1018D0008A011120063085000130870083165908DF
:1018E0008312A3008316580883128A011120063040
:1018F000850015308700831659088312A3008316CC
:10190000580883128A0111200330850017308700A0
:10191000831659088312A3008316580883128A017C
:101920001120043085008701831659088312A30013
:101930008316580883128A01112006308500013071
:101940008700831659088312A30083165808831250
:101950008A0111200730850024308700831659083A
:101960008312A3008316580883128A0111200730BE
:1019700085002B308700831659088312A300831635
:10198000580883128A011120073085002F30870004
:10199000831659088312A3008316580883128A01FC
:1019A000112008004630E000E10104308500870185
:1019B0006108A30060088A011120043085001030FE
:1019C00087006108A30060088A01112004308500A7
:1019D000113087006108A30060088A011120850189
:1019E00087016108A30060088A0111200430850086
:1019F00087016108A30060088A0111200630850074
:101A0000203087006108A30060088A011120063099
:101A100085002A3087006108A30060088A01112030
:101A2000063085002B3087006108A30060088A011A
:101A30001120850187016108A30060088A01112037
:101A40000430850087016108A30060088A01112025
:101A500006308500203087006108A30060088A01F5
:101A6000112007308500243087006108A30060083A
:101A70008A011120073085002E3087006108A300FD
:101A800060088A011120073085002F308700610827
:101A9000A30060088A011120850187016108A30065
:101AA00060088A01112008003230E200E3010130B1
:101AB000850087016308A30062088A01112085015F
:101AC00087016308A30062088A01112001308500A4
:101AD00087016308A30062088A0111208501103084
:101AE00087006308A30062088A011120850187012D
:101AF0006308A30062088A01112085011030870065
:101B00006308A30062088A01112085010430870060
:101B10006308A30062088A01112085018701630818
:101B2000A30062088A011120850104308700630840
:101B3000A30062088A011120013085008701630833
:101B4000A30062088A011120850187016308A300B0
:101B500062088A0111200130850087016308A30013
:101B600062088A011120023085000830870063086E
:101B7000A30062088A011120850187016308A30080
:101B800062088A011120023085000830870063084E
:101B9000A30062088A0111208501223087006308B2
:101BA000A30062088A011120850187016308A30050
:101BB00062088A0111208501223087006308A30092
:101BC00062088A0111208501043087006308A300A0
:101BD00062088A011120850187016308A300620859
:101BE0008A0111208501043087006308A300620880
:101BF0008A0111200130850087016308A300620873
:101C00008A011120850187016308A30062088A0107
:101C100011200130850087016308A30062088A0152
:101C2000112002308500083087006308A300620895
:101C30008A011120850187016308A30062088A01D7
:101C4000112002308500083087006308A300620875
:101C50008A01112004308500013087006308A30049
:101C600062088A011120850187016308A3006208C8
:101C70008A01112004308500013087006308A30029
:101C800062088A0111208501223087006308A300C1
:101C900062088A011120850187016308A300620898
:101CA0008A0111208501223087006308A3006208A1
:101CB0008A0111208501043087006308A3006208AF
:101CC0008A011120850187016308A30062088A0147
:101CD00011208501043087006308A30062088A018F
:101CE000112008003230E400E5010430850087014E
:101CF0006508A30064088A01112085018701650831
:101D0000A30064088A01112004308500870165085A
:101D1000A30064088A01112085011030870065083E
:101D2000A30064088A011120850187016508A300CA
:101D300064088A0111208501103087006508A3001E
:101D400064088A0111208501013087006508A3001D
:101D500064088A011120850187016508A3006408D1
:101D60008A0111208501013087006508A3006408FD
:101D70008A0111200430850087016508A3006408EA
:101D80008A011120850187016508A30064088A0182
:101D900011200430850087016508A30064088A01CA
:101DA000112002308500203087006508A3006408F8
:101DB0008A011120850187016508A30064088A0152
:101DC000112002308500203087006508A3006408D8
:101DD0008A01112085010A3087006508A300640884
:101DE0008A011120850187016508A30064088A0122
:101DF000112085010A3087006508A30064088A0164
:101E000011208501013087006508A30064088A015C
:101E10001120850187016508A30064088A0111204B
:101E20008501013087006508A30064088A0111203C
:101E30000430850087016508A30064088A01112029
:101E4000850187016508A30064088A011120043018
:101E5000850087016508A30064088A01112002300B
:101E60008500203087006508A30064088A011120DE
:101E7000850187016508A30064088A0111200230EA
:101E80008500203087006508A30064088A011120BE
:101E900001308500043087006508A30064088A01CA
:101EA0001120850187016508A30064088A011120BB
:101EB00001308500043087006508A30064088A01AA
:101EC000112085010A3087006508A30064088A0193
:101ED0001120850187016508A30064088A0111208B
:101EE00085010A3087006508A30064088A01112073
:101EF0008501013087006508A30064088A0111206C
:101F0000850187016508A30064088A011120850105
:101F1000013087006508A30064088A0111200800C9
:101F200004308500113087006708A30066088A0125
:101F300011208501283087006708A30066088A0100
:101F4000112001308500143087006708A30066085F
:101F50008A01112002308500023087006708A30043
:081F600066088A011120080047
:02400E00FC3F75
:00000001FF
